:02000000DA29FB
:1000080083120313FF00030E8301B8000A08B70028
:100018008A017008A6007408A5007808A4007A0868
:10002800A3007B08A2007C08A1007D08A000803006
:100038008F00B20A80303B3AF000803032067002FE
:1000480003185F28B201A80A80303B3AF0008030DC
:100058002806700203184D28A801B30A8030173A01
:10006800F00080303306700203183B28B3010A30D1
:10007800F4003308F0007D2130307007A9000A3001
:10008800F4003308F0007D217808F0003030700764
:10009800AA000A30F4002808F0007D2130307007EB
:1000A800AC000A30F4002808F0007D217808F00040
:1000B80030307007AD000A30F4003208F0007D21BE
:1000C80030307007AF000A30F4003208F0007D21AC
:1000D8007808F00030307007B0000130A7000C102D
:1000E8002608F0002508F4002408F8002308FA0080
:1000F8002208FB002108FC002008FD0037088A00C0
:0A010800380E8300FF0E7F0E090081
:0E011200213083120313FD00FD0B8D28080021
:06012000000000000800D1
:100126000F3083120313FC004730FD00FD0B9928A6
:0A013600FC0B9928000000000800EF
:1001400083120313BE1BA6288611A72886153E1B03
:10015000AB280611AC280615BE1AB0288610B128A7
:1001600086143E1AB5280512B62805163618BA2880
:100170000515BB280511851590208511BE19C228CB
:100180008611C32886153E19C7280611C8280615EA
:10019000BE18CC288610CD2886143E18D12805120A
:1001A000D22805163618D6280515D7280511851525
:1001B00090208511361CDE289320DF288920080036
:0E01C0008312031335088A00340882000800F9
:1001CE008312031336103D08BE00A020361408001B
:1001DE000129803083120313B9001429C030B900ED
:1001EE0014299430B9001429D430B9001429803060
:1001FE00B9001429831203133908013A0319F028A0
:10020E003908023A0319F5283908033A0319F82870
:10021E003908043A0319FB28FE283A03F00039087E
:10022E00F0077008B9007008BE00A0203610BC019F
:10023E003C083B078400000803192D293C083B07A6
:10024E0084000008BD00E720BC0A1F2936140800F0
:10025E0083160313851105110512861006118611DA
:10026E008312851105118611061186100512932031
:10027E0093209320861405168515902085119320C2
:10028E00851590208511932085159020851193203A
:10029E0005128515902085119320851590208511C6
:1002AE0086108615851590208511932086110516CA
:1002BE0085159020851105128515902085119320A6
:1002CE008515902085110516851590208511932092
:1002DE0005128515902085118615061586140516AE
:0C02EE008515902085119320361408001F
:1002FA0083120313FD01F801700803190034740610
:10030A00FA00FA1BFD09FB01F41F8D29F409F40A0E
:10031A00701C9129F009F00A70087404FA00FA1B9B
:10032A00B5297408F802F00D700DF80D7408F80775
:10033A00F00D0630FC00700DF80D74087018F80204
:10034A00701CF807F00DFC0BA029701CF8077B182D
:10035A00C329FD1F0034F009F00AF809F80A00342D
:10036A00F41FC029F01BBD297008F800F001AE295E
:10037A00F001F00A0034F009FB0A9629F80A740819
:10038A007802031DAE29F801F00AF01FAE29FF34E6
:02039A00080059
:10039C00E0208A110A128000840AB40A0319B50AF3
:0803AC00F003031DCE29080037
:1003B400013083120313A7003A30A8003130A9009A
:1003C4003130AA003A30AB003530AC003830AD00E3
:1003D4003A30AE003530AF003130B000B1013330C7
:1003E400B2000B30B300703083168F009B010330D2
:1003F4008500C03086002F210130BE00A0200C30C3
:10040400BE00A0200F309000C0308B000130831656
:100414008C00803083128F002708013A031D1A2AAA
:100424000130B9000530BA002930BB00EF20A70124
:10043400051C4D2A80308F00B201B30A8030173A70
:10044400F0008030330670020318292AB3010A3001
:10045400F4003308F0007D2130307007A9000A3021
:10046400F4003308F0007D217808F0003030700784
:10047400AA003030AF003030B0000230FB00023050
:10048400FC002130FD00FD0B452AFC0B452AFB0B2B
:10049400452A0130A700851C802A80308F00B201D4
:1004A400A80A80303B3AF000803028067002031816
:1004B4005C2AA8010A30F4002808F0007D213030BD
:1004C4007007AC000A30F4002808F0007D21780899
:1004D400F00030307007AD003030AF003030B00085
:1004E4000230FB000230FC002130FD00FD0B782AB5
:1004F400FC0B782AFB0B782A0130A7000E2A812AEC
:04400E00183F030054
:00000001FF
